:0200000022C01C
:10000200FECFFDCFFCCF70C0FACF4AC0F8CFF7CFFA
:10001200F6CFF5CFF4CFF3CFF2CFF1CFF0CFEFCFD2
:10002200EECFEDCF3F065B4F666D7D077F6F00E839
:100032000000000000000A00840026000800020000
:1000420030000000F894EE27ECBBE5BFF8E1A4B75E
:10005200A77FA4BFF1BDE1BD8DE0A2E0ED938A953B
:10006200E9F780E8A0E6ED938A95E9F7E8E3F0E0A6
:1000720085919591009761F0A591B59105901590A4
:10008200BF01F00105900D920197E1F7FB01F0CF5E
:10009200E0E0E3BBE4BBE5BBEFEDEDBFC0E84CC085
:1000A200AA93EA93FA93EFB7EA93EFEFE325E2BB61
:1000B200A0E8A90DEC91EC57E081E8BBE32DF0E05C
:1000C200F595E7953E2E9394E4E0E91519F4992409
:1000D200E8E03E2EE1E0E61509F4C798E991EFBFAA
:1000E200F991E991A9911895EA93EFB7EA93989B50
:1000F2001FC02394EAE0E21511F422245394EAE0AB
:10010200E51511F455244394EAE0E41511F444246E
:100112007394E6E0E71521F477247394E1E06E2E00
:1001220020928000E1E85082E2E84082E3E87082B7
:10013200E991EFBFE9911895E0E8E6BDE0E0E6BDA0
:10014200EBBBEABBE8BBEFEFE7BBEFE7E2BBEFE0FD
:10015200E1BBE0E0E0BFE3E0E3BFE0E0E2BFE4E018
:10016200E6BFE0E0ECBFEFBDEBE0EEBDE0E0EDBDF1
:10017200ECBDE5BDE4BDE4E0EBBDE2EEEABDE0E0EE
:10018200E9BDE8BDE2E4E9BFE0E8E8B9789419D056
:10019200E1E021D0E02141F0989A9998E0E06E2EBA
:1001A2007E2E4E2E5E2E2E2E0CD0E0E014D0E021BC
:1001B20011F0989A9998859902C09898999AE7CFE0
:1001C200FFCFA0E08699A1E0E0E005D00E2EA0E0EE
:1001D2009999A1E00895EA17E1E009F0EE27089560
:00000001FF
